:020000040800F2
:1000000000060220010200085D0F0008610F0008D1
:10001000B90F0008610F00088D0F000803020008E7
:10002000030200080302000803020008A5280008D4
:10003000030200080302000803020008030200088C
:10004000030200080302000803020008030200087C
:1000500003020008030200083D3A0008653A000860
:100060008D3A0008B53A0008DD3A0008030200089E
:10007000030200080302000803020008030200084C
:10008000030200080302000803020008030200083C
:10009000030200080302000803020008053B0008F1
:1000A000030200080302000803020008030200081C
:1000B000013C0008030200080302000803020008D4
:1000C00003020008030200080302000803020008FC
:1000D0000302000803020008D93B000803020008DD
:1000E000693B00080302000803020008030200083D
:1000F00003020008030200080302000803020008CC
:1001000003020008030200080302000803020008BB
:1001100003020008030200080302000803020008AB
:10012000030200080302000803020008030200089B
:10013000030200080302000803020008030200088B
:1001400003020008030200080302000879300008D7
:10015000030200080302000803020008030200086B
:10016000030200080302000803020008030200085B
:10017000030200080302000803020008030200084B
:100180000302000803020008ED3B00080302000818
:10019000030200080302000803020008030200082B
:1001A000030200080302000803020008030200081B
:1001B000030200080302000803020008030200080B
:1001C00003020008030200080302000803020008FB
:1001D00003020008030200080302000803020008EB
:1001E00003020008030200080302000803020008DB
:1001F00003020008030200080302000803020008CB
:1002000002E000F000F8FEE772B63A4880F3088892
:10021000394880F3098839484EF60851CEF200017A
:10022000086040F20000CCF200004EF63471CEF2CD
:1002300000010860BFF34F8FBFF36F8F40F20000E3
:10024000C0F2F0004EF68851CEF200010860BFF314
:100250004F8FBFF36F8F4FF00000E1EE100A4EF6A4
:100260003C71CEF200010860062080F31488BFF3D1
:100270006F8F02F0D9FB02F079FB03F075FA4FF0B3
:1002800055301F491B4A91423CBF41F8040BFAE725
:100290001C49194A91423CBF41F8040BFAE71A493C
:1002A0001A4A1B4B9A423EBF51F8040B42F8040B0A
:1002B000F8E700201749184A91423CBF41F8040B67
:1002C000FAE702F097FB03F0B9FA144C144DAC4274
:1002D00003DA54F8041B8847F9E700F041F8114CA1
:1002E000114DAC4203DA54F8041B8847F9E702F0D9
:1002F0007FBB000000060220002202200000000850
:1003000000000220000602204040000800220220D7
:100310006822022068220220E4360220000200083F
:100320000002000800020008000200082DE9F04F5A
:100330002DED108AC1F80CD0D0F80CD0BDEC108A8D
:10034000BDE8F08F002383F311882846A0470020E2
:1003500001F0CEFEFEE701F04FFE00DFFEE70000F9
:1003600038B500F0E7FC40B1174B6FF07F01002279
:1003700059720F211A729972DA7202F055FA044614
:1003800002F08AFA0546D0B9104B9C4219D00133CD
:100390009C4241F2883412BF05460024012500200A
:1003A00002F04CFA0DB100F05BF800F077FD00F0C0
:1003B00007FC204600F0F4F800F052F8F9E70024BA
:1003C000EDE70446EBE700BF00220220010007B082
:1003D00008B500F0C1FBA0F120035842584108BD08
:1003E000054B07B51B88022101A8ADF8043000F0C9
:1003F000D1FB03B05DF804FBB43C000810B520232A
:1004000083F311881248C3680BB101F0F9FE002391
:10041000104A4FF47A710E4801F0B4FE002383F3C2
:1004200011880D4C236813B12368013B2360636876
:1004300013B16368013B6360084B1B7833B9636891
:1004400023B9022000F092FC3223636010BD00BF8C
:1004500068220220FD030008842302207C2202205F
:10046000454B46492DE9F04153F8042F013201D1A3
:10047000BDE8F0818B42F7D1414C424B22689A4251
:1004800078D9414B9B6803F1006303F500439A421E
:1004900070D2002000F0AEFB02203C4B187000F040
:1004A00059FC3B4B1A6C00221A64196E1A66196EBD
:1004B000596C5A64596E5A66596E596941F08001F7
:1004C0005961596921F0800159615969196941F0EF
:1004D00000511961196921F0005119611B6972B647
:1004E0002C4B2D490B601D682468BFF34F8FBFF361
:1004F0006F8F2A4BC3F88420BFF34F8F5A6922F4C1
:1005000080325A61BFF34F8FD3F8802043F6E07EEC
:10051000C2F3C906C2F34E32B707520102EA0E080F
:1005200038463146013948EA000C00F14040B1F14B
:10053000FF3FC3F874C2F5D1203A12F1200FEDD17C
:10054000BFF34F8FBFF36F8FBFF34F8FBFF36F8F2B
:100550005A6922F400325A610022C3F85022BFF3D4
:100560004F8FBFF36F8F202383F31188AD4685F340
:1005700008882047BDE8F081FC7F00081C80000847
:1005800004800008FF7F0008002202207C22022055
:10059000003802400080000808ED00E000ED00E0B7
:1005A0002DE9F04F99B0BB4D2022FF21009010A8FB
:1005B000AC6800F015FCB84A01951378A3B9012185
:1005C000B6481170C360202383F31188C3680BB150
:1005D00001F016FE0023B24A4FF47A71AF4801F0E1
:1005E000D1FD002383F31188009BAE4A03B1136051
:1005F0000026AD4B009DB2463746B1461E70566090
:100600000293012000F0A6FB002D00F02B82A54BE9
:100610001B68002B40F0268219B0BDE8F08F022045
:10062000FFF7D6FE002840F01682009B02210BA89F
:10063000002E08BF1D469D4B1B88ADF82C3000F0E6
:10064000A9FADEE74FF47A7000F086FAB0F10008FC
:10065000EBDB0220FFF7BCFE0028E6D008F1FF38F4
:10066000B8F1050F00F2F981DFE808F0030B0E1175
:10067000143718A80523042140F8343D00F08AFA05
:1006800017E004218348F9E704218948F6E70421AB
:100690008848F3E74FF01C09484609F1040900F0C7
:1006A000ABFA04210B900BA800F074FAB9F12C0FEF
:1006B000F2D101234FF0000903FA08F848EA0A0AC8
:1006C0005FFA8AFA00F0E0FB27B10AF00B030B2B6C
:1006D00008BF0025FFF784FE93E704217648CDE7A5
:1006E000002FA2D00AF00B030B2B9ED10220FFF7A4
:1006F0006FFE8046002898D001206B4E00F07AFAF9
:1007000000270220307000F025FB5FFA87FB584677
:1007100000F080FA054688B15846013700F08AFAA1
:100720000028F2D146460025644B02210BA847461B
:100730001B88ADF82C3000F02DFA62E701232C461F
:100740000220337000F0F8FA019B9B689C4206D2AD
:10075000204600F051FA0130E4D10434F4E70024DB
:10076000029B464647461C7025464E4B5C60A9E7F7
:10077000002F3FF45AAF0AF00B030B2B7FF455AF59
:100780000220029B187000F0E5FA322000F0E4F934
:10079000B0F1000BFFF649AF1BF003087FF445AF43
:1007A000019B04EB0B0299688A423FF63EAFBBF512
:1007B000807F3FF63AAF424AD84503920FDA4FF4B2
:1007C0007A7000F0C9F9049004990029FFF62DAF62
:1007D0000499039A08F8021008F10108ECE7C82010
:1007E000FFF7F6FD804600283FF41FAF1F2C11D8FD
:1007F000C4F1200710AB24F0030031495F451844D1
:1008000028BF5F463A4600F0C3FA3A46FF212C481B
:1008100000F0E6FA4FEAAB0329492046DAB2039327
:1008200000F0E6FA074600283FF47EAF039B04EB96
:10083000830447E70220FFF7CBFD00283FF4F5AE25
:1008400000F01EFA00283FF4F0AE4FF000084346D7
:10085000019A9268904535D2B8F11F0F12D8109ABC
:1008600001320FD028F0030218A90A4452F8202CB4
:100870000B92184604220BA908F1040800F0B0FB03
:100880000346E5E74046039300F0B6F9039B0B905F
:10089000EFE700BF0022022080230220682202200E
:1008A000FD030008842302207C220220B63C0008BD
:1008B00004220220082202200C220220B83C000858
:1008C0008022022018A8042140F84C3D00F062F973
:1008D000F8E618A80023642140F8343D00F050F9F0
:1008E00000287FF4A2AE0220FFF772FD00283FF43B
:1008F0009CAE0B9800F0B0F918AB43F8480D0421FA
:100900001846E3E718A80023642140F8343D00F0BE
:1009100037F900287FF489AE0220FFF759FD00283F
:100920003FF483AE0B9800F0A5F918AB43F8440DE3
:10093000E5E70220FFF74CFD00283FF476AE00F01B
:10094000AFF918AB43F8400DD9E70220FFF740FD9F
:1009500000283FF46AAE0BA9142000F0A7F98046E6
:1009600018A8042140F83C8D00F014F941460BA86A
:10097000ACE7322000F0F0F8B0F10008FFF655AE19
:1009800018F0030F7FF451AE019A08EB0903926847
:1009900093423FF64AAE0220FFF71AFD00283FF4CB
:1009A00044AE28F00308C844C1453FF48BAE484626
:1009B00009F1040900F020F904210A900AA800F0C6
:1009C000E9F8F1E74FF47A70FFF702FD00283FF4F1
:1009D0002CAE00F055F9002842D0109B01330BD00B
:1009E000082210A9002000F003FA002838D02022A5
:1009F000FF2110A800F0F4F9FFF7F2FC3A4801F0EB
:100A00007DFB09E6002F3FF410AE0AF00B030B2B21
:100A10007FF40BAE18A80023642140F8343D00F0A9
:100A2000AFF8804600287FF400AE0220FFF7D0FC2C
:100A300000283FF4FAAD0390FFF7D2FC41F2883072
:100A4000454601F05BFB0B9800F068FA00F01CFAD9
:100A5000039B1F46D5E5074634E64FF00009E4E561
:100A6000B84661E6002000F077F80490049B002B64
:100A7000FFF6CAAD012000F05FF9049B213B162B65
:100A80003FF6BFAD01A252F823F000BF1F060008D9
:100A900045060008E10600080306000803060008F2
:100AA00003060008710700087309000835080008EC
:100AB000D3080008050900083309000803060008E8
:100AC0004B09000803060008C5090008C506000810
:100AD00003060008050A00082B060008C5060008E2
:100AE00003060008D3080008A08601002DE9F84F8E
:100AF0004FF47A7507460E4600245543DFF85080C0
:100B0000DFF8509098F900305FFA84FA5A1C01D04F
:100B1000A34210D159F82400324639460368D3F86D
:100B200020B02B46D847864205D1084B012083F8D8
:100B300000A0BDE8F88F0134032CE3D14FF4FA7024
:100B400001F0DCFA0020BDE8F88F00BFD0230220BE
:100B500010220220BC3C000807B5002202AB012194
:100B600003F8012D02461846FFF7C0FF20B19DF89B
:100B7000070003B05DF804FB4FF0FF30F9E7000019
:100B80000A46042108B5FFF7B1FF80F00100C0B2AA
:100B9000404208BD074B30B41A78074B53F8224047
:100BA0000A46014623682046DD69044BAC4630BC4A
:100BB000604700BFD0230220BC3C0008A086010093
:100BC00070B50A4C00250A4E01F034FD20803068D3
:100BD0002388834208D901F027FD33680544013397
:100BE000B5F5004F3360F2D370BD00BFD2230220B1
:100BF0008C23022001F0CABD00F1006000F5004026
:100C00000068704700F10060920000F5004001F0BC
:100C100057BD0000054B1A68054B1B889B1A834281
:100C200002D9104401F000BD002070478C2302203F
:100C3000D223022038B5074D04462868204401F02D
:100C4000FBFC28B928682044BDE8384001F00CBD01
:100C500038BD00BF8C23022010F0030308D1B0F58B
:100C6000846F05D200F10050A0F571200068704734
:100C700000207047014BC058704700BF20F4F01FA0
:100C8000064991F8243033B100230822086A81F81C
:100C90002430FFF7B7BF0120704700BF9023022028
:100CA000014B1868704700BF002004E01F4BF0B5EF
:100CB0001E681F4BC6F30B02360C1F885D68BA42D4
:100CC00093F9084022D09F89BA4221D01F8BBA42A3
:100CD00006D102220C2404FB02335D6893F908401C
:100CE000B6F5805F16D041F201039E4208BF5A2438
:100CF000421E013D0B460A44934215D215F9016F7D
:100D0000581C4EB1034600F8016CF5E70022E1E7FC
:100D10000122DFE74124EBE72C2582421D7001D937
:100D2000981C5C70401AF0BD1846FBE7002004E0F8
:100D30001422022000207047022804D14FF48002C0
:100D4000034B9A6170470128FCD14FF40002F7E78A
:100D500000080240022803D14022034B9A617047E9
:100D60000128FCD18022F8E700080240022805D1C2
:100D7000064A536983F04003536170470128FCD150
:100D8000024A536983F08003F6E700BF000802407F
:100D9000002310B5934203D0CC5CC4540133F9E76F
:100DA00010BD000030B5441E14F9010F0B4658B1B8
:100DB00093F900500131854206D11AB993F9002008
:100DC000801A30BD013AEFE7002AF7D1104630BD56
:100DD00002460346981A13F9011B0029FAD17047FD
:100DE00002440346934202D003F8011BFAE770471E
:100DF0002DE9F047234C05468846174694F82430E1
:100E000083BB2E46DFF87C90C7B394F824302BB90F
:100E10002022FF2148462662FFF7E2FF94F82400D3
:100E20004146C0F1080504EB8000BD4228BF3D46A5
:100E30005FFA85FAAD00A7EB0A072A462E44FFF7B2
:100E4000A7FF94F82430A844FFB29A445FFA8AFAC4
:100E5000BAF1080F84F824A0D6D1FFF711FF0028BB
:100E6000D2D108E0266A06EB8306B042CAD0FFF76B
:100E700007FF0028C5D10020BDE8F0870120BDE8AC
:100E8000F08700BF90230220024B1A78024B1A70A1
:100E9000704700BFD02302201022022038B5184C22
:100EA000184D204600F038FC2946204600F060FC32
:100EB0002D681548EA6ED2F8043843F00203C2F8F0
:100EC000043801F01BF91149284600F05FFDEA6E75
:100ED0000F48D2F804380F49A04223F00203C2F8A9
:100EE00004384FF4E1330B6001D000F073FB0A4883
:100EF000A04204D00749BDE8384000F06BBB38BDC4
:100F0000682A0220D83D000840420F00003E000839
:100F1000D4230220B82302204024022038B50B4BF2
:100F200005461A780A4B53F822400A4B9C420CD0D3
:100F3000094B002118221846FFF752FF05600146B1
:100F40002046BDE8384000F045BB38BDD023022024
:100F5000BC3C0008682A0220B8230220FEE70000FB
:100F600000B59BB0EFF3098168226846FFF710FFD8
:100F7000EFF30583044B9A6BDA6A9A6A9A6A9A6A63
:100F80009A6A9A6A9B6AFEE700ED00E000B59BB0A2
:100F9000EFF3098168226846FFF7FAFEEFF3058355
:100FA000044B9A6B9A6A9A6A9A6A9A6A9A6A9B6AD4
:100FB000FEE700BF00ED00E000B59BB0EFF3098154
:100FC00068226846FFF7E4FEEFF30583034B5A6B94
:100FD0009A6A9A6A9A6A9A6A9B6AFEE700ED00E04A
:100FE00030B50A44074D91420BD011F8013B09245A
:100FF0005840013CF7D040F300032B4083EA5000F7
:10100000F7E730BD2083B8ED026843681143016003
:1010100003B1184770470000024A136843F0C00349
:101020001360704700440040024A136843F0C00355
:10103000136070470078004037B51A4C1A4D2046AF
:1010400000F0BCFA009404F1140000234FF4807205
:10105000164900F07DF900944FF48072144904F1B0
:101060003800144B00F0F6F9134B2566E365134C7A
:10107000204600F0A3FA04F11400009400234FF47A
:1010800080720F4900F064F900940E4B4FF48072A7
:101090000D4904F1380000F0DDF90C4B2566E365DD
:1010A00003B030BDD423022080F93703AC240220E2
:1010B000AC26022019100008004400404024022001
:1010C000AC25022029100008AC270220007800403F
:1010D000284B002908BF1946037C012B30B50CD1E1
:1010E000254B984236D1254B1A6C42F400321A64D3
:1010F0001A6E42F400321A661B6E0A68036EC46DE3
:1011000003EB52038166B3FBF2F34A68150442BF56
:1011100023F0070503F0070343EA4503E3608B6808
:1011200043F040036360CB68510543F00103A360C3
:1011300042F4967343F0010323604FF0FF332362C0
:1011400005D512F0102211D0B2F1805F10D080F8D6
:10115000643030BD0A4B9842CFD1084B1A6C42F034
:1011600080421A641A6E42F08042C4E77F23EEE7A1
:101170003F23ECE7F43C0008D4230220003802406F
:10118000402402202DE9F047C66D05463768F46912
:10119000200734621AD014F0080F0CBF0021802100
:1011A000E20748BF41F02001A3074FF0200348BFEA
:1011B00041F04001600748BF41F4807183F311881A
:1011C000281DFFF721FF002383F31188E2050AD5CC
:1011D000202383F311884FF40071281DFFF714FFBB
:1011E000002383F311884FF020094FF0000A14F018
:1011F000200831D13B0616D54FF0200905F1380AF9
:10120000200610D589F31188504600F057F90028C0
:101210002FDA0821281DFFF7F7FE27F0800333603F
:10122000002383F3118879060DD562060BD52023A0
:1012300083F31188EA6C2B6D9A4201D12B6CEBB9C8
:10124000002383F31188E30620D5AA6E1369EBB15E
:101250005069BDE8F047184789F31188736A28463A
:1012600095F86410194000F0C3F98AF31188F46905
:10127000BDE7B06288F31188F469C1E727F0400741
:101280001021281DFFF7C0FE3760D9E7BDE8F087C1
:10129000F8B51546826804460B46AA4200D2856816
:1012A000A1692669761AB54207D218462A46FFF781
:1012B0006FFDA3692B44A3610DE011D9AF1B32462A
:1012C0001846FFF765FD3A46E1683044FFF760FDD8
:1012D000E2683A44A261A36828465B1BA360F8BD9C
:1012E00018462A46FFF754FDE368E4E78368934213
:1012F0002DE9F04104460F46154600D28568606925
:101300002669361AB54207D22A463946FFF740FD0C
:1013100063692B4463610EE013D9A5EB06083246DE
:101320003946FFF735FD4246B919E068FFF730FD51
:10133000E26842446261A36828465B1BA360BDE883
:10134000F0812A463946FFF723FDE368E2E7000013
:1013500010B50A440024C361029B006040608460B1
:10136000C160816141610261036210BD08B582699B
:101370004369934201D1826882B9826801328260F6
:101380005A1C42611970426903699A4201D3C368C9
:101390004361002100F0CEFE002008BD4FF0FF3079
:1013A00008BD000070B5202304460E4683F3118863
:1013B000A568A5B1A368A269013BA360531CA36102
:1013C00015782269934224BFE368A361E3690BB1F6
:1013D00020469847002383F31188284670BD314684
:1013E000204600F097FE0028E2DA85F3118870BDF0
:1013F0002DE9F74F05460F4690469A46D0F81C90C7
:10140000202686F311884FF0000B144664B1224663
:1014100039462846FFF73CFF034668B9514628463F
:1014200000F078FE0028F1D0002383F31188A8EBA8
:10143000040003B0BDE8F08FB9F1000F03D00190B4
:101440002846C847019B8BF31188E41A1F4486F392
:101450001188DBE7C160816141611144C361009B78
:10146000006040608260016103627047F8B5044625
:101470000E461746202383F31188A568A5B1A368FB
:10148000013BA36063695A1C62611E702369626933
:101490009A4224BFE3686361E3690BB12046984731
:1014A000002080F31188F8BD3946204600F032FE56
:1014B0000028E2DA85F31188F8BD000083694269EB
:1014C0009A4210B501D182687AB98268013282608D
:1014D0005A1C82611C7803699A4201D3C3688361F4
:1014E000002100F027FE204610BD4FF0FF3010BD58
:1014F0002DE9F74F05460F4690469A46D0F81C90C6
:10150000202686F311884FF0000B144664B1224662
:1015100039462846FFF7EAFE034668B95146284691
:1015200000F0F8FD0028F1D0002383F31188A8EB28
:10153000040003B0BDE8F08FB9F1000F03D00190B3
:101540002846C847019B8BF31188E41A1F4486F391
:101550001188DBE7026843681143016003B1184753
:10156000704700001430FFF743BF00004FF0FF3317
:101570001430FFF73DBF00003830FFF7B9BF00005F
:101580004FF0FF333830FFF7B3BF00001430FFF7E0
:1015900009BF00004FF0FF311430FFF703BF000018
:1015A0003830FFF763BF00004FF0FF323830FFF7ED
:1015B0005DBF000000207047FFF73EBD044B036095
:1015C000002343608360C36001230374704700BF3E
:1015D0000C3D000810B52023044683F31188FFF763
:1015E00077FD02232374002383F3118810BD0000CC
:1015F00038B5C36904460D461BB904210844FFF7FA
:10160000A9FF294604F11400FFF7B0FE002806DA0E
:10161000201D4FF48061BDE83840FFF79BBF38BD07
:10162000026843681143016003B118477047000026
:1016300013B5446BD4F8A4381A681178042915D16D
:10164000217C022912D11979012312898B4013427E
:101650000CD101A904F14C0001F08AFFD4F8A44890
:101660000246019B2179206800F0E0F902B010BD2C
:10167000143001F00DBF00004FF0FF33143001F0C3
:1016800007BF00004C3001F0DFBF00004FF0FF3318
:101690004C3001F0D9BF0000143001F0DBBE000077
:1016A0004FF0FF31143001F0D5BE00004C3001F096
:1016B000ABBF00004FF0FF324C3001F0A5BF00007F
:1016C000D0F8A42838B5136805461978042901D044
:1016D000012038BD017C0229FAD1527901205C89B0
:1016E00090400440F4D105F1140001F06DFE024673
:1016F0000028EDD0D5F8A4584FF480732868697994
:1017000000F082F9204638BD406BFFF7D9BF0000DA
:1017100000207047704700007FB5124B012504265A
:10172000044603600023057400F1840243602946E7
:101730008360C3600C4B0290143001934FF48073AC
:10174000009601F01DFE094B04F2944229460193D4
:1017500004F14C004FF480730294009601F0E4FE13
:1017600004B070BD343D00080917000831160008A8
:101770000B68202282F311880A7903EB820210623F
:101780004A790D3243F822008A7912B103EB8203C1
:1017900018620223C0F8A4180374002383F311888D
:1017A0007047000038B5037F044613B190F85430F9
:1017B000ABB90125201D0221FFF732FF04F114000F
:1017C00025776FF0010100F0C1FC84F8545004F15A
:1017D0004C006FF00101BDE8384000F0B7BC38BDE7
:1017E00010B5012104460430FFF71AFF00232377C8
:1017F00084F8543010BD000038B50446002514307C
:1018000001F0D6FD04F14C00257701F0A5FE201D66
:1018100084F854500121FFF703FF2046BDE838400B
:10182000FFF74EBF90F85C3003F06003202B19D116
:1018300090F85D20212A0AD0222A4FF000030ED012
:10184000202A0FD1084A02650722426504E0064BB0
:101850000365072343650023836501207047036503
:101860004365F9E70020704738220220D0F8A438F9
:1018700037B51A680446117804291AD1017C022967
:1018800017D11979012312898B40134211D100F12C
:101890004C05284601F020FF58B101A9284601F067
:1018A00067FED4F8A4480246019B2179206800F025
:1018B000BDF803B030BD000000EB8103F7B51C6A32
:1018C00005460E46F4B1202383F3118805EB860705
:1018D000201D08214C34FFF7A3FEFB685B691B68E1
:1018E00013B1204601F052FE01A9204601F040FE4E
:1018F000024648B1019B3146284600F097F8002384
:1019000083F3118803B0F0BDFB685A691268002A9E
:10191000F5D01B8A013B1340F1D105F15C02EAE7E7
:101920000D3138B550F82140DCB1202383F3118804
:10193000D4F8A4281368527903EB8203DB689B690F
:101940005D6845B104216018FFF76AFE294604F17D
:10195000140001F043FD2046FFF7B2FE002383F39D
:10196000118838BD7047000001F0D8B8012300F19C
:10197000240200F1380103700023436042F8043B65
:101980008A421361FAD103814381704738B5044616
:10199000202383F3118800254160C56005614561FE
:1019A0008561C561056201F0C9F80223237085F3E2
:1019B000118838BD70B500EB8103054650690E46AD
:1019C0001446DA6018B110220021FFF709FAA06965
:1019D00018B110220021FFF703FA31462846BDE86E
:1019E000704001F075B90000028902F00102028125
:1019F000428902F001024281002202614261826159
:101A0000C261026201F0F8B9F0B4012500EB810473
:101A100047898D40E4683D43A469458123600023E4
:101A2000A2606360F0BC01F013BA0000F0B40125BD
:101A300000EB810407898D40E4683D4364690581BA
:101A400023600023A2606360F0BC01F08DBA000047
:101A500070B50223002504460370A0F8645080F896
:101A6000665080F8675005814581C5600561456114
:101A70008561C561056280F84C5001F0C5F8636866
:101A80001B6823B129462046BDE87040184770BD49
:101A9000037880F868300523037043681B6810B52D
:101AA00004460BB10421984700232381638110BDB4
:101AB000436890F868201B6802700BB10521184735
:101AC0007047000090F84C3070B5044613B1002305
:101AD00080F84C3004F15C02204601F0AFF96368F5
:101AE0009B6863BB94F85C5015F0600615D194F8C0
:101AF0005D3005F07F0545EA032540F202339D4243
:101B000000F00E815BD8022D00F0DC803FD8002D64
:101B100000F08780012D00F0CF800021204601F0E9
:101B2000FBFB0021204601F0EDFB63681B6813B14D
:101B3000062120469847062384F84C3070BD204685
:101B400098470028CED094F8632094F8623043EA96
:101B50000223626D934238BF636594F95C30656D12
:101B6000002B4FF0200380F2FD80002D00F0EC8070
:101B7000092284F84C2083F311880021636D226DC3
:101B80002046FFF753FF002383F3118870BDB5F59E
:101B9000817F00F0B180B5F5407F49D0B5F5807FF9
:101BA000BBD194F85E30012BB7D1B4F8643023F088
:101BB0000203A4F8643026656665A665C3E740F2B3
:101BC00001639D421ED8B5F5C06F3BD2B5F5A06F3D
:101BD000A3D1B4F85C30B3F5A06F0ED194F85E30A9
:101BE000204684F8663001F067F863681B6813B11B
:101BF0000121204698470323237000232365636552
:101C0000A365A0E7B5F5106F32D040F602439D42C0
:101C100052D0B5F5006F80D104F16703236501232D
:101C200024E004F16403A5652365022363658AE764
:101C300094F85E30012B7FF470AFB4F8643043F059
:101C40000203B6E794F861202046616894F860309A
:101C50004D6843EA022394F85F1094F85E20A84789
:101C600000283FF45AAF4368236503686365A4E71F
:101C70002378042B10D1202383F311882046FFF70B
:101C8000B3FE86F311886368032184F867601B68DC
:101C900021700BB12046984794F85E30002BACD0F1
:101CA00084F867300423237063681B68002BA4D07A
:101CB000022120469847A0E7374B2365022363653E
:101CC00000239DE794F86010204611F0800F01F08A
:101CD0000F010ED001F0A4F8012806D002287FF4ED
:101CE0001CAF2E4B6065236567E72D4B656523654B
:101CF00063E701F087F8EFE794F85E30002B7FF49C
:101D00000CAF94F8603013F00F013FF476AF1A0671
:101D1000204602D501F014FB6FE701F007FB6CE7EA
:101D200094F85E30002B7FF4F8AE94F8603013F036
:101D30000F013FF462AF1B06204602D501F0ECFA1A
:101D40005BE701F0DFFA58E7142284F84C2083F3B4
:101D500011882B462A4629462046FFF755FE85F373
:101D6000118870BD5DB1152284F84C2083F3118871
:101D70000021636D226D2046FFF746FE03E70B222C
:101D800084F84C2083F311882B462A4629462046A6
:101D9000FFF74CFEE3E700BF643D00085C3D000830
:101DA000603D000838B590F84C300446152B29D812
:101DB000DFE803F03E28282828283E28280B293968
:101DC00028282828282828283E3E90F8631090F8D4
:101DD0006220436D42EA01229A4214D9C268128AF3
:101DE000B3FBF2F502FB15356DB9202383F311889F
:101DF0002B462A462946FFF719FE85F311880A2348
:101E000084F84C3038BD142384F84C30202383F3FD
:101E10001188002320461A461946FFF7F5FD0023D6
:101E200083F3118838BD836D03B198470023E7E73A
:101E3000002101F071FA0021204601F063FA636885
:101E40001B6813B10621204698470623D8E70000F7
:101E500090F84C20152A38B5044622D80123934027
:101E600040F6416213421DD113F480150FD19B023D
:101E700017D50B2380F84C30202383F311882B4691
:101E80002A462946FFF7D2FD85F3118838BDC3687D
:101E90009B695B682BB9836D03B19847002384F875
:101EA0004C3038BD002101F037FA0021204601F006
:101EB00029FA63681B6813B1062120469847062358
:101EC000EDE70000024B00221B605B609A607047E8
:101ED000AC280220002382680374054B1B689968B4
:101EE0009142FBD25A6803604260106058607047AC
:101EF000AC28022008B5202383F31188037C032B30
:101F000005D0042B0DD02BB983F3118808BD43698C
:101F100000221A604FF0FF334361FFF7DBFF00231D
:101F2000F2E790E80C001A6002685360F2E70000E4
:101F3000002382680374054B1B6899689142FBD8A3
:101F40005A6803604260106058607047AC280220F5
:101F5000054B196908741868026853601A601861A3
:101F600001230374FEF7E2B9AC2802204B1C30B504
:101F7000054687B00A4C10D0236901A8094A00F031
:101F800001F92846FFF7E4FF049B13B101A800F014
:101F900037F92369586907B030BDFFF7D9FFF8E773
:101FA000AC280220F51E000838B50C4D04464161EE
:101FB0002B6981689A68914203D8BDE83840FFF7E1
:101FC00089BF1846FFF7B4FF01232C610146237433
:101FD0002046BDE83840FEF7A9B900BFAC28022072
:101FE000044B1A681B6990689B68984294BF002054
:101FF00001207047AC28022010B5084C23682069E6
:102000001A6854602260012223611A74FFF790FF5E
:1020100001462069BDE81040FEF788B9AC280220CF
:10202000FEE7000010B50C4CFFF74CFF00F09CF8E9
:1020300080220A49204600F021F8012344F8180CB8
:10204000037400F03FFC002383F3118862B6044858
:10205000BDE8104000F034B8D4280220683D0008E4
:10206000703D000800F008B9034B59685A68521ACD
:102070009042FBD8704700BF001000E0826002224F
:1020800002740022427470478368A3F17C0243F813
:102090000C2C026943F83C2C426943F8382C074A5F
:1020A00043F81C2CC268A3F1180043F8102C02223C
:1020B00003F8082C002203F8072C7047450300089A
:1020C00010B5202383F31188FFF7DEFF00210446BB
:1020D000FFF76AFF002383F31188204610BD00003C
:1020E000024B1B6958610F20FFF732BFAC2802205A
:1020F000202383F31188FFF7F3BF000008B50146E2
:10210000202383F311880820FFF730FF002383F397
:10211000118808BD49B1064B42681B6918605A60B6
:10212000136043600420FFF721BF4FF0FF3070477A
:10213000AC2802200368984206D01A6802605060FA
:1021400018465961FFF7C6BE7047000038B504460F
:102150000D462068844200D138BD036823605C606E
:102160004561FFF7B7FEF4E7054B03F114025A612E
:102170009A614FF0FF32DA6100221A62704700BFA5
:10218000AC280220F8B503610E46C260054601F096
:10219000D7FA1A4B19461F4651F8142F8A420DD10F
:1021A00018620A2E2CBF80190A30AE606A602A605D
:1021B0009D615D61BDE8F84001F0B0BA1B6A9268AC
:1021C000C41A341928BF3446A24202D9181901F0A2
:1021D000B3FA7B699A6894420CD8AC6098685A68E4
:1021E000041B2B606A6015605D609C604FF0FF33DC
:1021F000FB61F8BDA41A1B68ECE700BFAC28022005
:1022000038B51C4B01685A691D4690420DD0446890
:102210002160002102685460C160916880680144B7
:1022200091604FF0FF32DA6138BD1A4642F8141F50
:102230004A6000215B69C160934203D1BDE8384028
:1022400001F074BA9A6881680A449A602C6A01F0B5
:1022500077FA6A69001B926882420AD9111A092921
:1022600098BF00F10A02286ABDE83840104401F026
:1022700063BA38BDAC2802202DE9F041184D002783
:1022800005F114066C6901F05BFA2A6AA368811AE9
:102290008B4216D81344D4F80C802B6294E80C00BF
:1022A0001A60226853606B69E760B34201D101F0A4
:1022B0003DFA87F311882069C047202383F31188F2
:1022C000E0E76A69B24208D05B1ABDE8F0410A2B28
:1022D0002CBFC0180A3001F02FBABDE8F08100BF52
:1022E000AC28022000207047FEE700007047000085
:1022F0004FF0FF3070470000022906D0032906D0B6
:102300000129064818BF0020704705487047032A76
:102310009ABF044800EBC200002070475C3E0008F2
:10232000103E00084822022070B59AB006460846C2
:10233000144601AD294600F0BDF82846FEF748FDD9
:10234000C0B2431C5B0086E81800237003230234EC
:1023500004F8013C00231946DAB20234904201D855
:102360001AB070BDEA5C013304F8011C04F8022CB9
:10237000F2E7000008B5202383F311880348FFF734
:1023800075FA002383F3118808BD00BF682A022074
:1023900090F85C3003F01F02012A07D190F85D200D
:1023A0000B2A03D100230365436512E003F06003A9
:1023B000202B11D1B0F8603073B990F85D20212A3C
:1023C00003D0222AEFD0202A06D1044A0265072230
:1023D0004265836501207047FFF724BA3F2202203F
:1023E00010B50446052916D8DFE801F016150316C6
:1023F000161D202383F311880E4A0121FFF7DAFA14
:1024000020460D4A0221FFF7D5FA0C48FFF7F4F9F0
:10241000002383F3118810BD202383F3118807481C
:10242000FFF7C0F9F4E7202383F311880348FFF78F
:10243000D7F9EDE7903D0008B43D0008682A022076
:1024400038B50C4D0C4C2A460C4904F10800FFF736
:102450006BFF05F1CA0204F110000949FFF764FFA0
:1024600005F5CA7204F118000649BDE83840FFF7C7
:102470005BBF00BF4033022048220220E03D00083D
:10248000EA3D0008F53D000870B5044608460D46D3
:10249000FEF79EFCC6B22046013403780BB91846FD
:1024A00070BD32462946FEF77DFC0028F3D101209D
:1024B00070BD00002DE9F04704460D46FEF788FC8C
:1024C0002B49C6B22046FFF7DFFF08B10A36F6B245
:1024D00028492046FFF7D8FF08B11036F6B2632E20
:1024E0000BD8DFF88C80DFF88C90234FDFF894A0B6
:1024F000267846B92E70BDE8F08721462846BDE80B
:10250000F04701F0CFBB252E2ED1072241462046B1
:10251000FEF748FC70B9194B2A4603F1100153F835
:10252000040B8B4242F8040BF9D11B7807341135A8
:102530001370DDE7082249462046FEF733FC98B9C0
:10254000AA1C0F4B13F8011F023209095345C95D3C
:1025500002F8041C197801F00F01C95D02F8031C90
:10256000F0D118350834C3E72E7001340135BFE7C8
:102570007C3E0008F53D0008963E0008843E0008B9
:102580001FF4F01F2BF4F01FBFF34F8F024AD368E4
:10259000DB03FCD4704700BF003C024008B5074B8A
:1025A0001B7853B9FFF7F0FF054B1A69002A04DACC
:1025B000044A5A6002F188325A6008BD9E350220F2
:1025C000003C02402301674508B5054B1B7833B931
:1025D000FFF7DAFF034A136943F00043136108BDB4
:1025E0009E350220003C02400B2870B513D80B4AE0
:1025F0000B4C137863B94FF000610A4E44F8231076
:1026000056F8235001330C2B2944F7D101231370C2
:1026100054F8200070BD002070BD00BFD0350220EE
:10262000A0350220A83E0008014B53F82000704757
:10263000A83E00080C2070470B2810B5044601D9AD
:10264000002010BDFFF7D0FF064B53F8243018448C
:10265000C21A0BB9012010BD12680132F0D1043B3F
:10266000F6E700BFA83E00080B2810B5044621D8A5
:10267000FFF78AFFFFF792FF0F4AF323D360C300EF
:10268000DBB243F4007343F002031361136943F4B4
:1026900080331361FFF778FFFFF7A6FF074B53F86E
:1026A000241000F0DBF8FFF78FFF2046BDE8104054
:1026B000FFF7C2BF002010BD003C0240A83E00084A
:1026C0002DE9F84312F0010315463FD18218B2F10B
:1026D000026F3BD22B4B1B6813F0010336D0FFF780
:1026E0005DFF294CF32340F20127E360FFF74CFF25
:1026F000032D01D9830712D00F46401A224C40F215
:102700000118EB1BC6190B44012B236924D823F0B5
:1027100001032361FFF758FF0120BDE8F883236917
:1027200023F44073236123693B43236151F8046B15
:102730000660BFF34F8FFFF727FF03689E4208D064
:10274000236923F001032361FFF73EFF0020BDE86A
:10275000F883043D0430CBE723F44073B94623618A
:10276000236943EA0803236137F8023B3380BFF350
:102770004F8FFFF709FF3688B6B2B9F80030B34281
:10278000BFD0DDE700380240003C0240084908B5F0
:102790000B7828B153B9FFF701FF01230B7008BD77
:1027A00023B10870BDE80840FFF70EBF08BD00BFA9
:1027B0009E35022002440439064BD2B210B5904235
:1027C00000D110BD441C00B253F8200041F8040FA2
:1027D000E0B2F4E750280040104B30B51C6F2404E1
:1027E00007D41C6F44F400741C671C6F44F400444D
:1027F0001C670B4C024404392368D2B243F4807343
:102800002360084B904200D130BD441C51F8045F56
:1028100000B243F82050E0B2F4E700BF00380240B5
:10282000007000405028004007B5012201A9002097
:10283000FFF7C0FF019803B05DF804FB13B5044631
:10284000FFF7F2FFA04206D002A90122002041F8C2
:10285000044DFFF7C1FF02B010BD00000144BFF3FB
:102860004F8F064B884204D3BFF34F8FBFF36F8F58
:102870007047C3F85C022030F4E700BF00ED00E0D1
:10288000034B1B689B0042BF0122024B1A7070472A
:1028900074380240D1350220014B1878704700BFD0
:1028A000D1350220EFF30983054968334A6822F0E5
:1028B00001024A6083F30988002383F3118870477B
:1028C00030EF00E0202080F3118862B60D4B0E4AF5
:1028D000D96821F4E0610904090C0A430B49DA6064
:1028E000CA6842F08072CA60094A0A49C2F8B01F39
:1028F000116841F0010111601022DA7783F822009B
:10290000704700BF00ED00E00003FA05F0ED00E0C5
:10291000001000E055CEACC510B5202383F311881C
:102920000E4B5B6813F4006314D0F1EE103AEFF332
:1029300009844FF08073683CE361094BDB682366D0
:1029400084F30988FFF74CFB10B1064BA36110BD5F
:10295000054BFBE783F3118810BD00BF00ED00E0DD
:1029600030EF00E0570300085A030008F0B5BFF34A
:102970004F8FBFF36F8F1D4B0021C3F85012BFF371
:102980004F8FBFF36F8F5A6942F400325A61BFF321
:102990004F8FBFF36F8FC3F88410BFF34F8FD3F8FF
:1029A000802043F6E076C2F3C904C2F34E32A50795
:1029B000520102EA060E284621464EEA0007013976
:1029C00000F14040C3F860724F1CF6D1203A12F17A
:1029D000200FEED1BFF34F8F5A6942F480325A6113
:1029E000BFF34F8FBFF36F8FF0BD00BF00ED00E06E
:1029F000FEE70000084A094B09498B4204D3094A03
:102A00000021934205D3704752F8040F43F8040B9A
:102A1000F3E743F8041BF4E7A4400008E43602207F
:102A2000E4360220E436022070470000036F0021E4
:102A300070B5C46E4FF0FF359E684A01A318D3F8F5
:102A40000009002805DAD3F8000940F08040C3F8F7
:102A50000009D3F8000B002805DAD3F8000B40F08A
:102A60008040C3F8000B0131A3188E42C3F8085907
:102A7000C3F8085BE1D24FF00113C4F81C3870BDF5
:102A8000890141F02001016103699B06FCD41220F9
:102A9000FFF7EABA204B03EB80022DE9F047D2F8AA
:102AA0000CE0461CDD6EDEF8142005EB0636D2F88D
:102AB00000C005EB4018516861450BD30123D5F8E0
:102AC000342803FA00F022EA0000C5F8340818465A
:102AD000BDE8F087ACEB0103BEF81040A34228BF6D
:102AE0002346D8F81849A4B2B3EB840F10D89468E1
:102AF0001F46A4F1040959F804AF042FC6F800A03A
:102B000001D9043FF7E71C440B4494605360D2E7BB
:102B10000020BDE8F08700BFD435022010B5054C79
:102B20002046FEF723FF4FF0A043E366024B2367E6
:102B300010BD00BFD4350220FC3E00080378012BF5
:102B400070B5054650D12A4BC46E98421BD1294B13
:102B50000E2143205A6B42F080025A635A6D42F0B4
:102B600080025A655A6D5A6942F080025A615A6968
:102B700022F080025A615B6900F0ECFB1E4BE360BF
:102B80001E4BC4F800380023EE6EC4F8003EC0238C
:102B900023604FF40413A3633369002BFCDA012391
:102BA0000C203361FFF760FA3369DB07FCD4122095
:102BB000FFF75AFA3369002BFCDA00262846A66094
:102BC000FFF734FF6B68C4F81068DB68C4F814685A
:102BD000C4F81C684BB90A4BA3614FF0FF33636123
:102BE000A36843F00103A36070BD064BF4E700BF88
:102BF000D435022000380240401400400300200277
:102C0000003C30C0083C30C0F8B5C46E0546002119
:102C10004FF000662046FFF733FF296F00234FF087
:102C200001128F684FF0FF30C4F83438C4F81C2804
:102C300004EB431201339F42C2F80069C2F8006BF3
:102C4000C2F80809C2F8080BF2D20B68EA6E6B678B
:102C5000636210231361166916F01006FBD112206F
:102C6000FFF702FAD4F8003823F4FE63C4F8003802
:102C7000A36943F4402343F01003A3610923C4F87C
:102C80001038C4F814380A4BEB604FF0C043C4F856
:102C9000103B084BC4F8003BC4F81069C4F8003975
:102CA0006B6F03F1100243F480136A67A362F8BDEF
:102CB000D83E000840800010C26E90F86610D2F82E
:102CC000003823F4FE6343EA0113C2F8003870476A
:102CD0002DE9F0410EB20D4600EB8608D8F80C1035
:102CE0000F6807F00303022B50D0032B50D03D4A4E
:102CF0003D4F012B18BF1746C46E4FEA451E0022F8
:102D000005F1100C04EB0E03C3F8102B8A69002A9E
:102D100040D04A8A05F158033A435B01E25001234F
:102D2000D4F81C2803FA0CF31343C4F81C38A64447
:102D300000234A69CEF8103905F13F03002A39D043
:102D40000A8A04EB8303898B9208012988BF4A43CE
:102D5000416F561841EA02422946466720465A60AA
:102D6000FFF78EFED8F80C301B8A43EA85531F43C9
:102D700005F148035B01E7500123D4F81C2803FA4E
:102D800005F51543C4F81C58BDE8F081174FB3E7AB
:102D9000174FB1E704EB4613D3F8002B22F400429F
:102DA000C3F8002B0123D4F81C2803FA0CF322EA01
:102DB0000303BAE704EB83030E4A04EB46162946E5
:102DC0005A602046FFF75CFED6F80039012223F452
:102DD000004302FA05F5C6F80039D4F81C3823EA96
:102DE0000505CFE700800010008004100080081067
:102DF00000800C1000040002026F12684267FFF7A7
:102E000015BE00005831C36E49015B5813F40040F1
:102E100004D013F4001F14BF0120022070470000EB
:102E20004831C36E49015B5813F4004004D013F4D9
:102E3000001F14BF012002207047000000EB810139
:102E4000CB68196A0B6813604B68536070470000C9
:102E500000EB810330B5DD68AA691368D36019B946
:102E6000402B84BF402313606B8A1468C26E1C44DD
:102E700002EB4110013C09B2B4FBF3F463430333AA
:102E800023F0030343EAC44343F0C043C0F8103BBC
:102E90002B6803F00303012B0ED1D2F8083802EBA4
:102EA000411013F4807FD0F8003B14BF43F08053EF
:102EB00043F00053C0F8003B02EB4112D2F8003B54
:102EC00043F00443C2F8003B30BD00002DE9F0415F
:102ED000244D0446EE6E06EB4013D3F8087B38070A
:102EE000C3F8087B0AD5D6F81438190706D505EBC0
:102EF000840321462846DB685B689847FA072FD58C
:102F0000D6F81438DB072BD505EB8403D968CCB988
:102F10008B69488A5E68B6FBF0F200FB12628AB9E0
:102F20001868DA6890420DD2121A83E81400202340
:102F300083F311880B482146FFF78AFF84F3118839
:102F4000BDE8F081012303FA04F26B8923EA02034E
:102F50006B81CB6823B121460248BDE8F041184798
:102F6000BDE8F081D435022000EB81034A0170B541
:102F7000DD68C36E6C692668E66056BB1A444FF480
:102F80000020C2F810092A6802F00302012A0AB2DE
:102F90000ED1D3F8080803EB421410F4807FD4F864
:102FA000000914BF40F0805040F00050C4F8000900
:102FB00003EB4212D2F8000940F00440C2F80009C5
:102FC0000122D3F8340802FA01F10143C3F834189E
:102FD00070BD19B9402E84BF4020206020681A447B
:102FE0002E8A841940F00050013CB4FBF6F440EA0C
:102FF000C440C6E7F8B504461E48C56E05EB441349
:10300000D3F80869F107C3F8086917D5D5F810385F
:10301000DA0713D500EB8403D9684B691F68DA68B7
:10302000974218D2D21B00271A605F60202383F3D7
:1030300011882146FFF798FF87F31188330617D5CB
:103040000123D5F83428A340134211D02046BDE80F
:10305000F840FFF71FBD012303FA04F2038923EAB6
:10306000020303818B68002BE8D021469847E5E7EF
:10307000F8BD00BFD4350220A1482DE9F84FC56E38
:1030800004466E69AB691E4016F4805F6E6105D020
:10309000FEF7DEFCBDE8F84FFFF73EBC002E12DA6B
:1030A000D5F8003E9B0705D0D5F8003E23F003037A
:1030B000C5F8003ED5F80438914823F00103C5F85F
:1030C0000438FEF7F5FC370505D58D48FFF7AEFC53
:1030D0008B48FEF7DDFCB0040CD5D5F8083813F0AA
:1030E000060FEB6823F470530CBF43F4105343F402
:1030F000A053EB60310704D56368DB680BB18048EF
:103100009847F2026FD4B3020CD5D4F86C80002734
:103110004FF00109DFF8E8A1236FF9B29B688B42F9
:1031200080F09C80F70619D5E16E0A6AC2F30A178F
:1031300002F00F0302F4F012B2F5802F00F0B58018
:10314000B2F5402F0AD104EB830301F58051DB680F
:10315000186A00231A469F4240F09C803303D5F83A
:1031600018481DD5E70302D50020FFF7AFFEA503E1
:1031700002D50120FFF7AAFE600302D50220FFF767
:10318000A5FE210302D50320FFF7A0FEE20202D52F
:103190000420FFF79BFEA30202D50520FFF796FE51
:1031A00077037FF577AFE60702D50020FFF722FF10
:1031B000A50702D50120FFF71DFF600702D50220F9
:1031C000FFF718FF210702D50320FFF713FFE206E0
:1031D00002D50420FFF70EFFA3067FF55BAF0520A5
:1031E000FFF708FF56E7D4F86C8000274FF001097D
:1031F000DFF80CA1236F5FFA87FB9B685B4582D3E6
:1032000008EB4B13D3F8002902F44022B2F5802FCB
:1032100022D1D3F80029002A1EDAD3F8002942F07F
:103220009042C3F80029D3F80029002AFBDB594655
:10323000E06EFFF725FC228909FA0BF322EA03036B
:10324000238104EB8B03DB689B6813B1594650461E
:1032500098475846FFF71EFC0137CBE708EB4112B1
:10326000D2F8003B03F44023B3F5802F10D1D2F8FD
:10327000003B002B0CDA628909FA01F322EA03030E
:10328000638104EB8103DB68DB680BB15046984730
:10329000013741E79C0700D10A68072B03F10103BE
:1032A0009EBF0270120A013055E7023301F58051CA
:1032B00004EB8302526890690268D0F808C0406845
:1032C000A2EB000E0022104697420AD104EB8304C1
:1032D00063689B699A683A449A605A6817445F60C9
:1032E0003CE712F0030F00D10868964502F1010295
:1032F00082BF8CF80000000A0CF1010CE4E700BF6B
:10330000D4350220C36E03EB4111D1F8003B43F4E6
:103310000013C1F8003B7047C36E03EB4111D1F8B5
:10332000003943F40013C1F800397047C36E03EB52
:103330004111D1F8003B23F40013C1F8003B704762
:10334000C36E03EB4111D1F8003923F40013C1F827
:103350000039704700F1604300F01F020901400985
:1033600003F56143C9B2800083F80013012300F123
:103370006040934000F56140C0F8803103607047C1
:1033800030B50433039C0172002104FB0325C361A3
:10339000049B00600363059B4060C1604261026161
:1033A0008561046242628162C162436330BD000094
:1033B0000022416AC260416101616FF001018262D5
:1033C000C262FEF7C3BE000003694269934203D1A3
:1033D000C2680AB100207047181D70470369196060
:1033E0000021C2680132C260C269134482699342FB
:1033F000036124BF436A0361FEF79CBE38B50446EF
:103400000D46E3683BB162690020131D1268A36298
:103410001344E36238BD237A33B929462046FEF7C8
:1034200079FE0028EDDA38BD6FF00100FBE70000FF
:10343000C368C269013BC360436913448269934214
:10344000436124BF436A436100238362036B03B17A
:103450001847704770B52023044683F31188866AA5
:103460003EB9FFF7CBFF054618B186F31188284611
:1034700070BDA36AE26A13F8015B9342A36202D3B0
:103480002046FFF7D5FF002383F31188EFE7000004
:103490002DE9F84F04460E4690469946202787F3BB
:1034A00011880025AA46D4F828B0BBF1000F09D135
:1034B00049462046FFF7A2FF20B18BF3118828462A
:1034C000BDE8F88FA16AA8EB050BE36A5B1A9B4580
:1034D00028BF9B46BBF1400F1BD9334601F1400288
:1034E00051F8040B914243F8040BF9D1A36A40361A
:1034F00040354033A362A26AE36A9A4202D320466F
:10350000FFF796FF8AF311884545D8D287F31188D3
:10351000C9E730465A46FDF73BFCA36A5E445D446A
:103520005B44A362E7E7000010B5029C043301721C
:10353000C36103FB0421002300608362C362039B19
:1035400040600363049BC460426102618161046264
:103550004262436310BD0000026A6FF00101C26065
:10356000426A4261026100228262C262FEF7EEBDDF
:10357000436902699A4203D1C2680AB100207047C8
:10358000184650F8043B0B6070470000C3680021E8
:10359000C2690133C3604369134482699342436142
:1035A00024BF436A4361FEF7C5BD000038B5044639
:1035B0000D46E3683BB1236900201A1DA262E2694F
:1035C0001344E36238BD237A33B929462046FEF717
:1035D000A1FD0028EDDA38BD6FF00100FBE7000027
:1035E00003691960C268013AC260C2691344826902
:1035F0009342036124BF436A036100238362036B28
:1036000003B118477047000070B5202304460E46EA
:1036100083F31188856A35B91146FFF7C7FF10B1EA
:1036200085F3118870BDA36A1E70A36AE26A013334
:103630009342A36204D3E16920460439FFF7D0FF27
:10364000002080F3118870BD2DE9F84F04460D4627
:1036500091469A464FF0200888F311880026B34619
:10366000A76A4FB951462046FFF7A0FF20B187F364
:1036700011883046BDE8F88FA06AA9EB0603E76A17
:103680003F1A9F4228BF1F46402F1BD905F1400318
:1036900055F8042B9D4240F8042BF9D1A36A40361B
:1036A0004033A362A26AE36A9A4204D3E1692046E6
:1036B0000439FFF795FF8BF311884E45D9D288F373
:1036C0001188CDE729463A46FDF762FBA36A3D44DF
:1036D0003E443B44A362E5E7026943699A4203D151
:1036E000C3681BB9184670470023FBE7836A002BA9
:1036F000F8D0043B9B1AF5D01360C368013BC3604C
:10370000C3691A4483699A42026124BF436A036110
:10371000002383620123E5E700F09EB84FF0804369
:10372000002258631A610222DA60704700224FF0CB
:103730008043DA60704700004FF080435863704761
:103740004FF08043586A70474B6843608B688360D2
:10375000CB68C3600B6943614B6903628B69436249
:103760000B6803607047000008B5274B40F2FF71FB
:1037700026481A690A431A611A6922F4FF6222F084
:1037800007021A611A691A6B0A431A631A6D0A430F
:103790001A651F4A1B6D1146FFF7D6FF1D4802F13F
:1037A0001C01FFF7D1FF1C4802F13801FFF7CCFFE5
:1037B0001A4802F15401FFF7C7FF194802F17001DE
:1037C000FFF7C2FF174802F18C01FFF7BDFF164853
:1037D00002F1A801FFF7B8FF144802F1C401FFF796
:1037E000B3FF134802F1E001FFF7AEFF114802F109
:1037F000FC01FFF7A9FF104802F58C71FFF7A4FF49
:10380000BDE8084000F09EB80038024000000240C9
:10381000083F00080004024000080240000C02407B
:10382000001002400014024000180240001C024038
:1038300000200240002402400028024008B500F0A9
:1038400013FAFEF7EFFBFFF71BF8BDE80840FEF7A1
:10385000F7BD0000704700000F4B1A6C42F00102E8
:103860001A641A6E42F001021A660C4A1B6E9368C3
:1038700043F0010393604FF080436B229A624FF054
:10388000FF32DA6200229A615A63DA605A600122DA
:103890005A611A60704700BF00380240002004E0FF
:1038A0004FF0804208B51369D1680B40D9B29B072D
:1038B0006FEA0101116107D5202383F31188FEF718
:1038C000D1FB002383F3118808BD00001B4B4FF090
:1038D000FF3000211A696FEA42526FEA52521A61B0
:1038E0001A69C2F30A021A611A695A6958615A6957
:1038F00059615A691A6A62F080521A621A6A02F0B1
:1039000080521A621A6A5A6A58625A6A59625A6A24
:103910000B4A106840F480701060186F00F440701B
:10392000B0F5007F03D04FF48030186719675368F3
:1039300023F40073536000F06BB900BF00380240FD
:1039400000700040374B4FF44041374A1A64374A01
:1039500011601A6842F001021A601A689207FCD5D9
:103960009A6822F003029A602E4B19469A6812F068
:103970000C02FBD1186800F0F90018609A601A6810
:1039800042F480321A600B689B03FCD54B6F43F006
:1039900001034B67234B5A6F9007FCD5244A5A60AA
:1039A0001A6842F080721A60204B1A46596849041E
:1039B000FCD5196841F4803119605368D803FCD5EF
:1039C000136843F400331360184A53689903FCD515
:1039D000144B1A689201FCD5164A9A6040F2011203
:1039E000C3F88C200022C3F8902040F20732124B1B
:1039F0001A601A6802F00F02072AFAD1094B9A6876
:103A000042F002029A609A6802F00C02082AFAD187
:103A10005A6C42F480425A645A6E42F480425A66AA
:103A20005B6E7047003802400004001000700040D8
:103A30000836400900948838003C0240074A08B51F
:103A4000536903F00103536123B1054A13680BB1B5
:103A500050689847BDE80840FEF75EBF003C014053
:103A600064360220074A08B5536903F00203536124
:103A700023B1054A93680BB1D0689847BDE8084068
:103A8000FEF74ABF003C014064360220074A08B5F1
:103A9000536903F00403536123B1054A13690BB161
:103AA00050699847BDE80840FEF736BF003C01402A
:103AB00064360220074A08B5536903F008035361CE
:103AC00023B1054A93690BB1D0699847BDE8084016
:103AD000FEF722BF003C014064360220074A08B5C9
:103AE000536903F01003536123B1054A136A0BB104
:103AF000506A9847BDE80840FEF70EBF003C014001
:103B000064360220164B10B55C6904F478725A6171
:103B1000A30604D5134A936A0BB1D06A984760068E
:103B200004D5104A136B0BB1506B9847210604D58E
:103B30000C4A936B0BB1D06B9847E20504D5094A48
:103B4000136C0BB1506C9847A30504D5054A936CD0
:103B50000BB1D06C9847BDE81040FEF7DDBE00BF4A
:103B6000003C014064360220194B10B55C6904F436
:103B70007C425A61620504D5164A136D0BB1506D33
:103B80009847230504D5134A936D0BB1D06D984720
:103B9000E00404D50F4A136E0BB1506E9847A10490
:103BA00004D50C4A936E0BB1D06E9847620404D5CD
:103BB000084A136F0BB1506F9847230404D5054A88
:103BC000936F0BB1D06F9847BDE81040FEF7A4BECD
:103BD000003C01406436022008B50348FDF7D2FAE4
:103BE000BDE80840FEF798BED423022008B503487C
:103BF000FDF7C8FABDE80840FEF78EBE402402205B
:103C000008B5FFF74DFEBDE80840FEF785BE000091
:103C1000062108B50846FFF79DFB06210720FFF7A0
:103C200099FB06210820FFF795FB06210920FFF7E5
:103C300091FB06210A20FFF78DFB06211720FFF7D5
:103C400089FB06212820FFF785FB07211C20FFF7B1
:103C500081FB0C212620FFF77DFB0C215220BDE8C3
:103C60000840FFF777BB000008B5FFF72FFE00F014
:103C70000DF8FDF7A1FCFDF777FEFDF74BFDFFF713
:103C8000E9FDBDE80840FFF747BD000000230449F7
:103C90001A465A50C81808334260802BF9D1704731
:103CA00064360220034611F8012B03F8012B002A89
:103CB000F9D170471210121312110000682A022065
:103CC000D42302204024022053544D3332463F3F38
:103CD0003F3F3F3F0053544D333246375B347C35D2
:103CE0005D780053544D333246375B367C375D7810
:103CF000000000000096000000000000000000002E
:103D000000000000000000000000000000000000B3
:103D1000811500086D150008A91500089515000803
:103D2000A11500088D150008791500086515000813
:103D3000B5150008000000008D160008791600086F
:103D4000B5160008A1160008AD160008991600085F
:103D50008516000871160008111700080000000001
:103D600001000000000000006D61696E00000000AD
:103D7000883D0008F0280220682A02200100000087
:103D8000212000080000000069646C65000000004C
:103D90000200000000000000B91800082119000806
:103DA00040004000103302202033022002000000B7
:103DB000000000000300000000000000651900087A
:103DC000000000001000000030330220000000005E
:103DD0000100000000000000D435022001010200B3
:103DE0004172647550696C6F740025424F415244B2
:103DF000252D424C002553455249414C25000000D9
:103E0000E1230008F9220008912300087523000827
:103E100043000000183E000809024300020100C0F0
:103E2000320904000001020201000524001001050E
:103E30002401000104240202052406000107058272
:103E4000030800FF09040100020A00000007050141
:103E5000024000000705810240000000120000003F
:103E6000643E00081201100102000040091241578F
:103E700000020102030100000403090425424F412E
:103E8000524425004355415676354E616E6F2D6282
:103E90006473686F740030313233343536373839F3
:103EA000414243444546000000800000008000007D
:103EB00000800000008000000000020000000400FC
:103EC00000000400000004000000040000000400E2
:103ED000000004000000040000000000C51A0008F3
:103EE000A51D0008511E0008400040004C3602206D
:103EF0004C360220010000005C36022080000000E9
:103F000040010000050000000000802A00000000C1
:103F1000AAAAAAAA00000000FFFF000000000000FB
:103F200000A00A000000000000000000AAAAAAAA3F
:103F300000000000FFFF0000000000000000000083
:103F40000050000000000000AAAAAAAA0000000079
:103F5000FFFF0000000000000000000080290000BA
:103F600000000000AAAAAAAA40150000FFFF000056
:103F70000070700700000000400002000000000018
:103F8000AAAAAAAA00000100F7FF00000000000092
:103F9000080000000020000000000000AAAAAAAA51
:103FA00000100000FFFF00000000000800000000FB
:103FB0000000000000000000AAAAAAAA0000000059
:103FC000FFFF0000000000000000000000000000F3
:103FD00000000000AAAAAAAA00000000FFFF00003B
:103FE00000000000000000000000000000000000D1
:103FF000AAAAAAAA00000000FFFF0000000000001B
:1040000000000000000000000000000000000000B0
:1040100000000000000000000000000000000000A0
:104020000000000000000000000000000000000090
:104030000000000000000000000000000000000080
:10404000320000000000000000801F00000000009F
:10405000FF00000000000000C83C00083F00000016
:1040600049040000D53C00083F0000005104000056
:10407000E33C00083F00000000960000000008003C
:10408000960000000008000004000000783E0008D0
:104090000000000000000000000000000000000020
:0840A000000000000000000018
:00000001FF
